:020000040000FA
:0400000096EF11F076
:080008006BEF0FF0D9CFE5FF0B
:10001000E1CFD9FF00C0E5FF01C0E5FF02C0E5FF69
:1000200003C0E5FF04C0E5FF05C0E5FF06C0E5FF2E
:1000300007C0E5FF08C0E5FF09C0E5FF0AC0E5FF0E
:100040000BC0E5FF0CC0E5FF0DC0E5FF0EC0E5FFEE
:100050000FC0E5FF10C0E5FF11C0E5FF12C0E5FFCE
:1000600013C0E5FF14C0E5FF020EDBCF00F0030E66
:10007000DBCF01F0040EDBCF02F0050EDBCF03F087
:10008000060EDBCF04F0070EDBCF05F0080EDBCF4A
:1000900006F0090EDBCF07F00A0EDBCF08F00B0EDF
:1000A000DBCF09F00C0EDBCF0AF00D0EDBCF0BF02F
:1000B0000001AD6B60AE29D0A49074AE13D009C01E
:1000C000E9FF0AC0F3FF0B506BEC11F00C6E0C86CD
:1000D0000CC0E5FF09C0E9FF0AC0F3FF0B50AEEC0E
:1000E00011F0749E0C6A60B00C2A0C50010BF46E77
:1000F0000001AD51FE0BF4100001AD6F0F0E0D6E3F
:10010000600E0C6E800E0E6E40D00F0150AF3BD0D3
:10011000A49274AC13D009C0E9FF0AC0F3FF0B50DE
:100120006BEC11F00F6E0F860FC0E5FF09C0E9FF01
:100130000AC0F3FF0B50AEEC11F0749C070E0F01D8
:1001400050150F6E0F500001AD6FADC0E8FF020EED
:100150000F5C12E209C0E9FF0AC0F3FF0B506BEC21
:1001600011F00F6E0F8E0FC0E5FF09C0E9FF0AC046
:10017000F3FF0B50AEEC11F00F0E0D6E500E0C6E27
:10018000800E0E6E02D0E86AFFD00CC00FF00DC0DA
:1001900010F00EC011F0000EE56E09C0E9FF0AC0B4
:1001A000F3FF0B50AEEC11F00C50050F126E000E69
:1001B0000D20136E000E0E20146E12C0E9FF13C046
:1001C000F3FF14506BEC11F0126E12500001AE6F81
:1001D000AEC0E8FF0F0E121612C0E5FF06C0E9FF21
:1001E00007C0F3FF0850AEEC11F00001AEAD12D025
:1001F00009C0E9FF0AC0F3FF0B506BEC11F0126E5F
:10020000128C12C0E5FF09C0E9FF0AC0F3FF0B50D2
:10021000AEEC11F00C50020F126E000E0D20136E9A
:10022000000E0E20146E12C0E9FF13C0F3FF14502D
:100230006BEC11F0126E12500001AE6F0001AEA710
:1002400016D009C0E9FF0AC0F3FF0B506BEC11F0A8
:10025000126E128A12C0E5FF09C0E9FF0AC0F3FF5F
:100260000B50AEEC11F0010E0001AE6F02D0000198
:10027000AE6B0C50010F126E000E0D20136E000EAF
:100280000E20146E0001AE51E56E0250E56E015075
:10029000E56E0050E56E1450E56E1350E56E125099
:1002A000E56E4BEC05F0070EE126060E0C26000E5F
:1002B0000D22000E0E2206C0E9FF07C0F3FF085012
:1002C0006BEC11F0066E06500001AE6F0CC000F032
:1002D0000DC001F00EC002F0066A06C007F0086A01
:1002E00006BE0868AEC00CF00D6A0850800FF36EB1
:1002F0000D50800FF35C02E10C50075C1DE200C062
:10030000E9FF01C0F3FF02506BEC11F0076E002A09
:10031000D8B0012AD8B0022A07C0E5FF03C0E9FF20
:1003200004C0F3FF0550AEEC11F0032AD8B0042A44
:10033000D8B0052A062AD1D7A4AE13D009C0E9FF48
:100340000AC0F3FF0B506BEC11F0006E008800C088
:10035000E5FF09C0E9FF0AC0F3FF0B50AEEC11F056
:10036000A49E0FC0E9FF10C0F3FF11506BEC11F019
:10037000006E009E00C0E5FF0FC0E9FF10C0F3FF54
:100380001150AEEC11F0010EE4CF14F0E4CF13F0F5
:10039000E4CF12F0E4CF11F0E4CF10F0E4CF0FF08F
:1003A000E4CF0EF0E4CF0DF0E4CF0CF0E4CF0BF08F
:1003B000E4CF0AF0E4CF09F0E4CF08F0E4CF07F08F
:1003C000E4CF06F0E4CF05F0E4CF04F0E4CF03F08F
:1003D000E4CF02F0E4CF01F0E4CF00F0E4CFD9FFA6
:1003E0001200D9CFE5FFE1CFD9FF00C0E5FF01C082
:1003F000E5FF02C0E5FF03C0E5FF04C0E5FF05C05F
:10040000E5FF06C0E5FF07C0E5FF08C0E5FF09C03E
:10041000E5FF0AC0E5FF0BC0E5FF0CC0E5FF0DC01E
:10042000E5FF0EC0E5FF0FC0E5FF020EDBCF00F0D9
:10043000030EDBCF01F0040EDBCF02F0800EE56E81
:1004400013EC11F0E12A0F0E046E180E036E800EED
:10045000056E000EE56E000EE56E000EE56E070EF1
:10046000E56EFF0EE56E0550E56E0450E56E035037
:10047000E56E0FEC08F0080EE1260F0E046E1C0E60
:10048000036E800E056E000EE56E000EE56E000E2A
:10049000E56E070EE56EFF0EE56E0550E56E045045
:1004A000E56E0350E56E0FEC08F0080EE126036AD6
:1004B000046A056A066A0450800F800F02E1060E86
:1004C000035CD8B04BD105500024076E06500120C4
:1004D000086EE86A06BEE8680220096E07C0E9FFF8
:1004E00008C0F3FF09502FEC11F0076EF3CF08F0AE
:1004F0000750FF0A04E10850FF0A01E12FD1830EE3
:100500000324096E000E04200A6E09C0E9FF0AC028
:10051000EAFFEFCF09F0060E095CD8B0F9D010C0A1
:10052000E5FF11C0E5FF116A09341136E8341136D0
:10053000FC0B106E000EFB6E050EFA6E540E1026AC
:100540001150FA22D8B0FB2A1050E4CF11F0E4CFBA
:1005500010F0F96EB6EF02F0D9EF02F0FCEF02F006
:100560001FEF03F042EF03F065EF03F00D01D481BC
:100570000F0E0A6E000E096E800E0B6E07C00CF097
:1005800008C00DF00E6A0F6A000EE56E0F50E56EA2
:100590000E50E56E0D50E56E0C50E56E0B50E56E9D
:1005A0000A50E56E0950E56E0FEC08F0080EE126E2
:1005B000CDD00D01D4830F0E0A6E040E096E800E8D
:1005C0000B6E07C00CF008C00DF00E6A0F6A000E2B
:1005D000E56E0F50E56E0E50E56E0D50E56E0C5059
:1005E000E56E0B50E56E0A50E56E0950E56E0FECB6
:1005F00008F0080EE126AAD00D01D4850F0E0A6E70
:10060000080E096E800E0B6E07C00CF008C00DF0CE
:100610000E6A0F6A000EE56E0F50E56E0E50E56E25
:100620000D50E56E0C50E56E0B50E56E0A50E56E10
:100630000950E56E0FEC08F0080EE12687D00D0199
:10064000D4870F0E0A6E0C0E096E800E0B6E07C05B
:100650000CF008C00DF00E6A0F6A000EE56E0F5028
:10066000E56E0E50E56E0D50E56E0C50E56E0B50CC
:10067000E56E0A50E56E0950E56E0FEC08F0080EC5
:10068000E12664D00D01D4890F0E0A6E100E096E9A
:10069000800E0B6E07C00CF008C00DF00E6A0F6ADA
:1006A000000EE56E0F50E56E0E50E56E0D50E56ED6
:1006B0000C50E56E0B50E56E0A50E56E0950E56E84
:1006C0000FEC08F0080EE12641D00D01D48B0F0E7F
:1006D0000A6E140E096E800E0B6E07C00CF008C077
:1006E0000DF00E6A0F6A000EE56E0F50E56E0E50AB
:1006F000E56E0D50E56E0C50E56E0B50E56E0A5040
:10070000E56E0950E56E0FEC08F0080EE1261ED0EC
:100710000D01D48B0F0E0A6E140E096E800E0B6E37
:100720000C6A0D6A000EE56E0D50E56E0C50E56E1C
:100730000850E56E0750E56E0B50E56E0A50E56E09
:100740000950E56E0FEC08F0080EE126020E0526B2
:10075000D8B0062A032AD8B0042AADD6000EE56E1A
:1007600013EC11F0E12AF36AE86AE4CF0FF0E4CF6A
:100770000EF0E4CF0DF0E4CF0CF0E4CF0BF0E4CFBB
:100780000AF0E4CF09F0E4CF08F0E4CF07F0E4CFBB
:1007900006F0E4CF05F0E4CF04F0E4CF03F0E4CFBB
:1007A00002F0E4CF01F0E4CF00F0E4CFD9FF120073
:1007B000D9CFE5FFE1CFD9FF00C0E5FF01C0E5FFDC
:1007C00002C0E5FF03C0E5FF04C0E5FF05C0E5FF8B
:1007D00006C0E5FF07C0E5FF08C0E5FF09C0E5FF6B
:1007E0000AC0E5FF0BC0E5FF0CC0E5FF0DC0E5FF4B
:1007F0000EC0E5FF0FC0E5FF10C0E5FF11C0E5FF2B
:1008000012C0E5FF13C0E5FF14C0E5FF15C0E5FF0A
:10081000020EDBCF00F0030EDBCF01F0040EDBCFC6
:1008200002F0050EDBCF03F0060EDBCF04F0070E5F
:10083000DBCF05F0080EDBCF06F0090EDBCF07F0AB
:100840000A0EDBCF08F00F0E0A6E400E096E800E06
:100850000B6E09500001606F0A500001616F0B5070
:100860000001626F0F0E0A6E300E096E800E0B6E65
:1008700009500001636F0A500001646F0B500001C2
:10088000656F0F0E0A6E200E096E800E0B6E0950FA
:100890000001666F0A500001676F0B500001686F1E
:1008A000096A0A6A020E095CD8B0C5D0600E0A2433
:1008B0000B6E0C6A000E0C220BC0E9FF0CC0EAFFA5
:1008C000EECF0BF0EECF0CF0EFCF0DF00BC00EF033
:1008D0000CC00FF00DC010F00BC0E9FF0CC0F3FF0F
:1008E0000D506BEC11F0116E11B6A1D0FC0E11166B
:1008F00011C0E5FF0BC0E9FF0CC0F3FF0D50AEECDB
:1009000011F00BC0E9FF0CC0F3FF0D506BEC11F0C0
:10091000116E030E0814126E1250111211C0E5FF71
:100920000BC0E9FF0CC0F3FF0D50AEEC11F008ACAA
:1009300004D0400E0710116E02D007C011F00B500A
:10094000050F126E000E0C20136E000E0D20146E9B
:1009500011C0E5FF12C0E9FF13C0F3FF1450AEEC65
:1009600011F008AA03D0010E116E01D0116A0B50CC
:10097000010F126E000E0C20136E000E0D20146E6F
:100980001150E56E0350E56E0250E56E0150E56EC4
:100990000050E56E1450E56E1350E56E1250E56E92
:1009A0000FEC08F0080EE126060E0B26000E0C22B6
:1009B000000E0D2204C011F005C012F006C013F0A5
:1009C000146A0750145C1DE211C0E9FF12C0F3FF66
:1009D00013506BEC11F0156E112AD8B0122AD8B052
:1009E000132A15C0E5FF0BC0E9FF0CC0F3FF0D5043
:1009F000AEEC11F00B2AD8B00C2AD8B00D2A142A6C
:100A0000E0D70EC0E9FF0FC0F3FF10506BEC11F000
:100A10000B6E0BB40AD00B860BC0E5FF0EC0E9FFCE
:100A20000FC0F3FF1050AEEC11F0010E05D0030E15
:100A30000A26092A37D7E86AE4CF15F0E4CF14F084
:100A4000E4CF13F0E4CF12F0E4CF11F0E4CF10F0D4
:100A5000E4CF0FF0E4CF0EF0E4CF0DF0E4CF0CF0D4
:100A6000E4CF0BF0E4CF0AF0E4CF09F0E4CF08F0D4
:100A7000E4CF07F0E4CF06F0E4CF05F0E4CF04F0D4
:100A8000E4CF03F0E4CF02F0E4CF01F0E4CF00F0D4
:100A9000E4CFD9FF1200D9CFE5FFE1CFD9FF00C0E5
:100AA000E5FF01C0E5FF02C0E5FF03C0E5FF04C0AC
:100AB000E5FF05C0E5FF06C0E5FF07C0E5FF08C08C
:100AC000E5FF09C0E5FF0AC0E5FF0BC0E5FF0CC06C
:100AD000E5FF0DC0E5FF020EDBCF00F0030EDBCF1C
:100AE00001F0040EDBCF02F0050EDBCF03F0060EA3
:100AF000DBCF04F0070EDBCF05F0080EDBCF06F0EE
:100B00000650D8A46CD000C0E9FF01C0F3FF02502A
:100B10006BEC11F0066E0638E840F80B076E07C064
:100B2000E5FF03C0E9FF04C0F3FF0550AEEC11F090
:100B30000350010F086E000E0420096E000E052000
:100B40000A6E0638E840070B066E06C0E5FF08C0CF
:100B5000E9FF09C0F3FF0A50AEEC11F0002AD8B04B
:100B6000012AD8B0022A00C0E9FF01C0F3FF0250F9
:100B70006BEC11F0066E0638E840070B066E065067
:100B8000071207C0E5FF03C0E9FF04C0F3FF0550EB
:100B9000AEEC11F00350020F066E000E0420076E3B
:100BA000000E0520086E000EE56E06C0E9FF07C0C6
:100BB000F3FF0850AEEC11F00350030F066E000E69
:100BC0000420076E000E0520086E000EE56E06C0BC
:100BD000E9FF07C0F3FF0850AEEC11F0A5D00350B9
:100BE000020F066E000E0420076E000E0520086E30
:100BF00000C0E9FF01C0F3FF02506BEC11F0096E79
:100C00000938E844E00B0A6E0AC0E5FF06C0E9FFB8
:100C100007C0F3FF0850AEEC11F00350030F0B6E4A
:100C2000000E04200C6E000E05200D6E0938E844FD
:100C30001F0B096E09C0E5FF0BC0E9FF0CC0F3FFF5
:100C40000D50AEEC11F0002AD8B0012AD8B0022A1B
:100C500006C0E9FF07C0F3FF08506BEC11F0E86E27
:100C600000C0E9FF01C0F3FF02506BEC11F0096E08
:100C7000030E09140B6E0B500A120AC0E5FF06C0E2
:100C8000E9FF07C0F3FF0850AEEC11F006C0E9FF22
:100C900007C0F3FF08506BEC11F0E86EE00E091688
:100CA0000938E8441F0B096E09500A120AC0E5FF13
:100CB00006C0E9FF07C0F3FF0850AEEC11F0002AB0
:100CC000D8B0012AD8B0022A0350010F066E000ED8
:100CD0000420076E000E0520086E00C0E9FF01C069
:100CE000F3FF02506BEC11F0096E09C0E5FF06C07E
:100CF000E9FF07C0F3FF0850AEEC11F0002AD8B0AE
:100D0000012AD8B0022A00C0E9FF01C0F3FF025057
:100D10006BEC11F0006E00C0E5FF03C0E9FF04C0FA
:100D2000F3FF0550AEEC11F0E4CF0DF0E4CF0CF082
:100D3000E4CF0BF0E4CF0AF0E4CF09F0E4CF08F001
:100D4000E4CF07F0E4CF06F0E4CF05F0E4CF04F001
:100D5000E4CF03F0E4CF02F0E4CF01F0E4CF00F001
:100D6000E4CFD9FF1200D9CFE5FFE1CFD9FF00C012
:100D7000E5FF01C0E5FF02C0E5FF03C0E5FF04C0D9
:100D8000E5FF05C0E5FF06C0E5FF07C0E5FF08C0B9
:100D9000E5FF09C0E5FF0AC0E5FF0BC0E5FF0CC099
:100DA000E5FF020EDBCF00F0030EDBCF01F0040EF7
:100DB000DBCF02F0050EDBCF03F0060EDBCF04F035
:100DC00000500110D8A4E6D002C0E9FF03C0F3FF31
:100DD00004502FEC11F0056EF3CF06F0000E065C08
:100DE00002E10A0E055CD8B057D00DC0E5FF0EC079
:100DF000E5FF0E6A05340E36E8340E36FC0B0D6E38
:100E0000000EFB6E0E0EFA6E200E0D260E50FA220C
:100E1000D8B0FB2A0D50E4CF0EF0E4CF0DF0F96E00
:100E200024EF07F028EF07F02CEF07F030EF07F082
:100E300034EF07F038EF07F03CEF07F040EF07F032
:100E400044EF07F048EF07F0010E056E066A27D061
:100E5000020E056E066A23D0040E056E066A1FD0C8
:100E6000080E056E066A1BD0100E056E066A17D0B6
:100E7000200E056E066A13D0400E056E066A0FD06E
:100E8000800E056E066A0BD0C00E056E066A07D08E
:100E9000056A010E066E03D0C00E056E066AB8869E
:100EA0000650E56E0550E56E020EE56E580EE56ED5
:100EB000FEEC0DF0076EF3CF08F0040EE126096A90
:100EC0000A6A2D0E0826310E0922010E0A2206504A
:100ED000E56E0550E56E010EE56E2C0EE56EFEEC3E
:100EE0000DF0056EF3CF06F0040EE1260B6A0C6AD6
:100EF0000C50E56E0B50E56E0650E56E0550E56E44
:100F00000A50E56E0950E56E0850E56E0750E56E33
:100F100059EC09F0056EF3CF06F0F4CF07F0E9CFF6
:100F200008F0080EE126000EE56E000EE56E000EDC
:100F3000E56E040EE56E0850E56E0750E56E06504E
:100F4000E56E0550E56E59EC09F0056EF3CF06F03D
:100F5000F4CF07F0E9CF08F0080EE126FF0E0526D2
:100F6000FF0E0622FF0E0722FF0E08220650E56E36
:100F70000550E56E3C0E28EC0FF0020EE1260E0E39
:100F8000C0EC11F0AB8EAB880F0EC0EC11F0F36A21
:100F9000010E28D00050010A02E1015001E020D0EA
:100FA000040E0226000E0322000E042202C0E9FFF6
:100FB00003C0F3FF04506BEC11F0026E025007E027
:100FC000949A94889496C76A210EC66E06D0949A15
:100FD00094889486C76A250EC66EF36A010E02D005
:100FE000F36AE86AE4CF0CF0E4CF0BF0E4CF0AF048
:100FF000E4CF09F0E4CF08F0E4CF07F0E4CF06F047
:10100000E4CF05F0E4CF04F0E4CF03F0E4CF02F046
:10101000E4CF01F0E4CF00F0E4CFD9FF1200D9CF44
:10102000E5FFE1CFD9FF00C0E5FF01C0E5FF02C049
:10103000E5FF03C0E5FF04C0E5FF05C0E5FF06C00E
:10104000E5FF07C0E5FF08C0E5FF09C0E5FF0AC0EE
:10105000E5FF020EDBCF00F0030EDBCF01F0040E44
:10106000DBCF02F0050EDBCFA0F0060EDBCFA1F048
:10107000070EDBCFA2F0080EDBCFA3F0090EDBCF0B
:1010800003F0000E056EA00E046E800E066E035077
:10109000D8A450D004C0E9FF05C0F3FF06506BECA4
:1010A00011F0036E0338E8441F0B076E07C0E5FF1D
:1010B00000C0E9FF01C0F3FF0250AEEC11F000C028
:1010C000E9FF01C0F3FF02506BEC11F0076E045012
:1010D000010F086E000E0520096E000E06200A6E34
:1010E00008C0E9FF09C0F3FF0A506BEC11F0086E6D
:1010F0000838E844E00B096E0950071207C0E5FF05
:1011000000C0E9FF01C0F3FF0250AEEC11F0002A6D
:10111000D8B0012AD8B0022A0338E844E00B076EA1
:1011200007C0E5FF00C0E9FF01C0F3FF0250AEECCD
:1011300011F0A6D00450020F036E000E0520076EBA
:10114000000E0620086E03C0E9FF07C0F3FF085039
:101150006BEC11F0036E0338E840070B076E07C015
:10116000E5FF00C0E9FF01C0F3FF0250AEEC11F053
:1011700000C0E9FF01C0F3FF02506BEC11F0076EF5
:101180000450030F086E000E0520096E000E0620A5
:101190000A6E08C0E9FF09C0F3FF0A506BEC11F0BA
:1011A000086E0838E840F80B096E0950071207C0AE
:1011B000E5FF00C0E9FF01C0F3FF0250AEEC11F003
:1011C000002AD8B0012AD8B0022A0338E840F80B28
:1011D000076EE00E071607C0E5FF00C0E9FF01C07B
:1011E000F3FF0250AEEC11F0078607C0E5FF00C028
:1011F000E9FF01C0F3FF0250AEEC11F0030E03163D
:101200000350071207C0E5FF00C0E9FF01C0F3FF6C
:101210000250AEEC11F0002AD8B0012AD8B0022A50
:101220000450010F036E000E0520076E000E06200D
:10123000086E03C0E9FF07C0F3FF08506BEC11F024
:10124000036E03C0E5FF00C0E9FF01C0F3FF0250D9
:10125000AEEC11F0002AD8B0012AD8B0022A04C09E
:10126000E9FF05C0F3FF06506BEC11F0046E04C0FB
:10127000E5FF00C0E9FF01C0F3FF0250AEEC11F042
:10128000E4CF0AF0E4CF09F0E4CF08F0E4CF07F0B0
:10129000E4CF06F0E4CF05F0E4CF04F0E4CF03F0B0
:1012A000E4CF02F0E4CF01F0E4CF00F0E4CFD9FFC7
:1012B0001200D9CFE5FFE1CFD9FF00C0E5FF01C0A3
:1012C000E5FF02C0E5FF03C0E5FF04C0E5FF05C080
:1012D000E5FF06C0E5FF07C0E5FF08C0E5FF09C060
:1012E000E5FF0AC0E5FF0BC0E5FF0CC0E5FF0DC040
:1012F000E5FF020EDBCF00F0030EDBCF01F0040EA2
:10130000DBCF02F0050EDBCF03F0060EDBCF04F0DF
:10131000070EDBCF05F0080EDBCF06F0090EDBCFA2
:1013200007F0D88003AED890086A083608500FE05E
:10133000031C0C6E021C0B6E011C0A6E001C096E55
:10134000092A0DE10A2A0BE10B4A0C2A08D000C039
:1013500009F001C00AF002C00BF003C00CF009C094
:1013600000F00AC001F00BC002F00CC003F0D880FE
:1013700007AED890096A093609500FE0071C0D6EB8
:10138000061C0C6E051C0B6E041C0A6E0A2A0DE16D
:101390000B2A0BE10C4A0D2A08D004C00AF005C044
:1013A0000BF006C00CF007C00DF00D50E56E0C50B0
:1013B000E56E0B50E56E0A50E56E0350E56E025087
:1013C000E56E0150E56E0050E56EB5EC0BF0006E79
:1013D000F3CF01F0F4CF02F0E9CF03F0080EE126DD
:1013E0000950081A085016E0031C076E021C066E0E
:1013F000011C056E001C046E042A04E1052A02E1AA
:10140000064A072A07C0E9FF06C0F4FF05C0F3FF3C
:10141000045007D003C0E9FF02C0F4FF01C0F3FF8E
:101420000050E4CF0DF0E4CF0CF0E4CF0BF0E4CFAC
:101430000AF0E4CF09F0E4CF08F0E4CF07F0E4CFFE
:1014400006F0E4CF05F0E4CF04F0E4CF03F0E4CFFE
:1014500002F0E4CF01F0E4CF00F0E4CFD9FF1200B6
:10146000D9CFE5FFE1CFD9FF00C0E5FF01C0E5FF1F
:1014700002C0E5FF03C0E5FF04C0E5FF05C0E5FFCE
:1014800006C0E5FF07C0E5FF08C0E5FF09C0E5FFAE
:101490000AC0E5FF0BC0E5FF0CC0E5FF0DC0E5FF8E
:1014A0000EC0E5FF020EDBCF00F0030EDBCF01F034
:1014B000040EDBCF02F0000E046E9C0E036E800E55
:1014C000056E0050030F066E000E0120076E000E21
:1014D0000220086E0050020F096E000E01200A6EF5
:1014E000000E02200B6E000E0D6EAC0E0C6E800E08
:1014F0000E6E0E50E56E0D50E56E0C50E56E0B5005
:10150000E56E0A50E56E0950E56E0850E56E07502D
:10151000E56E0650E56E0550E56E0450E56E03502D
:10152000E56E06EC00F0036E0C0EE126035003E1BD
:10153000F36AE86A42D000019C51036E00019D519C
:10154000046E03C0E5FF04C0F4FF00C0E9FF01C062
:10155000F3FF0250A2EC11F099C003F0032A0350EC
:101560000001996F0001AC51600B09E09BC003F0D2
:10157000032A035000019B6FF368E8681ED0000146
:10158000ACA709D09AC003F0032A035000019A6F58
:10159000F368FE0E12D0020E0026000E0122000E8D
:1015A000022200C0E9FF01C0F3FF02506BEC11F012
:1015B000006E016A01C0F3FF0050E4CF0EF0E4CFEB
:1015C0000DF0E4CF0CF0E4CF0BF0E4CF0AF0E4CF61
:1015D00009F0E4CF08F0E4CF07F0E4CF06F0E4CF61
:1015E00005F0E4CF04F0E4CF03F0E4CF02F0E4CF61
:1015F00001F0E4CF00F0E4CFD9FF12000001A46BAA
:10160000060E0001A56F020E00018B6F00018C6BAE
:10161000010E00018E6F010E0001956F000E016E2C
:101620008B0E006E800E026E0250E56E0150E56E6C
:101630000050E56E000EE56E000EE56EB3EC06F0B0
:10164000050EE126000E016E910E006E800E026EF8
:101650000250E56E0150E56E0050E56E000EE56E3D
:10166000010EE56EB3EC06F0050EE126000E016EEC
:10167000A40E006E800E026E0250E56E0150E56E03
:101680000050E56E000EE56E4AEC0DF0040EE1260A
:101690008AEC11F0FC0E93168A828A90006A016A25
:1016A000010E026E036A000EE56E010EE56EA2ECFD
:1016B00010F0046E020EE126045015E0000EE56EF7
:1016C000010EE56E75EC10F00001896F020EE12647
:1016D00000018951E56E000EE56E000EE56E42ECEC
:1016E00010F0030EE1260050980A03E101503A0A77
:1016F00001E00AD0DD0EE56E000EE56E000EE56E2F
:1017000042EC10F0030EE126000EE56E000EE56ED1
:10171000A2EC10F0046E020EE1260450010A13E15F
:10172000000EE56E000EE56E75EC10F0046E020E14
:10173000E1260450E56E000EE56E010EE56E42EC0A
:1017400010F0030EE126002AD8B0012A022AD8B0F0
:10175000032A0350800F460F02E1990E025C02E358
:101760008A80A1D78A909FD71200D9CFE5FFE1CF19
:10177000D9FF00C0E5FF01C0E5FF02C0E5FF03C0DF
:10178000E5FF04C0E5FF05C0E5FF06C0E5FF07C0B3
:10179000E5FF08C0E5FF09C0E5FF0AC0E5FF0BC093
:1017A000E5FF0CC0E5FF0DC0E5FF020EDBCF00F04A
:1017B000030EDBCF01F0040EDBCF02F0050EDBCF12
:1017C00003F0060EDBCF04F0070EDBCF05F0080EAA
:1017D000DBCF06F0090EDBCF07F0086A096A0A6A58
:1017E0000B6A200E0C6E0344010B0D6E010E0D16DC
:1017F0000050002601360236033608500826093606
:101800000A360B360D50D8A4088007500B5C08E14F
:1018100006500A5C05E10550095C02E10450085CD1
:1018200009E30450085E0550095A06500A5A075049
:101830000B5A00800C2ED7D703C0E9FF02C0F4FF7B
:1018400001C0F3FF0050E4CF0DF0E4CF0CF0E4CF83
:101850000BF0E4CF0AF0E4CF09F0E4CF08F0E4CFD6
:1018600007F0E4CF06F0E4CF05F0E4CF04F0E4CFD6
:1018700003F0E4CF02F0E4CF01F0E4CF00F0E4CFD6
:10188000D9FF1200D9CFE5FFE1CFD9FF00C0E5FFB6
:1018900001C0E5FF02C0E5FF03C0E5FF04C0E5FFAE
:1018A00005C0E5FF06C0E5FF07C0E5FF08C0E5FF8E
:1018B00009C0E5FF020EDBCF00F0030EDBCF01F025
:1018C000040EDBCF02F000C0E9FF01C0F3FF0250BD
:1018D0002FEC11F0036EF3CF04F0056A066A005096
:1018E000030F076E000E0120086E000E0220096E25
:1018F000020E0026000E0122000E022200C0E9FFA7
:1019000001C0F3FF02506BEC11F0006E000EE56EAB
:101910000050E56E0950E56E0850E56E0750E56E23
:101920000650E56E0550E56E0450E56E0350E56E19
:10193000D8EC03F0006E090EE126016A0050011098
:1019400007E097C002F0022A02500001976F06D00C
:1019500098C002F0022A02500001986F01C0F3FF04
:101960000050E4CF09F0E4CF08F0E4CF07F0E4CF73
:1019700006F0E4CF05F0E4CF04F0E4CF03F0E4CFC9
:1019800002F0E4CF01F0E4CF00F0E4CFD9FF120081
:10199000D9CFE5FFE1CFD9FF00C0E5FF01C0E5FFEA
:1019A00002C0E5FF03C0E5FF04C0E5FF05C0E5FF99
:1019B00006C0E5FF07C0E5FF08C0E5FF09C0E5FF79
:1019C0000AC0E5FF0BC0E5FF020EDBCF00F0030EFF
:1019D000DBCF01F0040EDBCF02F0050EDBCF03F00E
:1019E000060EDBCF04F0070EDBCF05F0080EDBCFD1
:1019F00006F00050011006E00050010A02E101501B
:101A000001E02DD0076A086A0850800FF36E065077
:101A1000800FF35C02E10550075C21E207500224CD
:101A2000096E085003200A6EE86A08BEE8680420C0
:101A30000B6E09C0E9FF0AC0F3FF0B506BEC11F00D
:101A4000096E0950E56E0150E56E0050E56E42ECFE
:101A500010F0030EE126072AD8B0082AD5D7E4CF24
:101A60000BF0E4CF0AF0E4CF09F0E4CF08F0E4CFC4
:101A700007F0E4CF06F0E4CF05F0E4CF04F0E4CFC4
:101A800003F0E4CF02F0E4CF01F0E4CF00F0E4CFC4
:101A9000D9FF1200D9CFE5FFE1CFD9FF00C0E5FFA4
:101AA00001C0E5FF02C0E5FF03C0E5FF020EDBCF8A
:101AB00000F0030EDBCF01F0040EDBCF02F0050EC9
:101AC000DBCF03F0030E005CD8B03CD004C0E5FFD0
:101AD00005C0E5FF056A00340536E8340536FC0B21
:101AE000046E000EFB6E1B0EFA6E020E04260550ED
:101AF000FA22D8B0FB2A0450E4CF05F0E4CF04F07A
:101B0000F96E87EF0DF0A2EF0DF0A2EF0DF0012AB4
:101B1000D8B0022AD8B0032A01C0E9FF02C0F3FFFF
:101B200003506BEC11F0006E080E005C09E2D56A00
:101B3000800ED510016E00500110D56E010E03D03D
:101B4000E86A01D0E86AE4CF03F0E4CF02F0E4CF22
:101B500001F0E4CF00F0E4CFD9FF1200D9CFE5FFC8
:101B6000E1CFD9FF00C0E5FF01C0E5FF02C0E5FFFE
:101B700003C0E5FF04C0E5FF05C0E5FF06C0E5FFC3
:101B800007C0E5FF020EDBCF00F0030EDBCF01F054
:101B9000040EDBCF02F0050EDBCF03F0060EDBCF29
:101BA00004F0056A0450055C15E205500024066E39
:101BB00001C0E9FF02C0F3FF03506BEC11F0076EA8
:101BC0000750E56E0650E56EA3EC0FF0020EE1261D
:101BD000052AE8D70450E4CF07F0E4CF06F0E4CFBD
:101BE00005F0E4CF04F0E4CF03F0E4CF02F0E4CF5B
:101BF00001F0E4CF00F0E4CFD9FF1200D9CFE5FF28
:101C0000E1CFD9FF00C0E5FF01C0E5FF02C0E5FF5D
:101C100003C0E5FF020EDBCF00F0030EDBCF01F0C7
:101C2000040EDBCF02F0050EDBCF03F00050000105
:101C3000A66F0150A76F02500001A86F0350A96F53
:101C40000001A6510001A803F3CF00F0F4CF01F08A
:101C500000500001AA6F0150AB6F0001A6510001B6
:101C6000A903F3CF00F00001A7510001A803F3CFAF
:101C700001F0015000260001AB5100260050AB6F6F
:101C8000ABC0F3FFAA51E4CF03F0E4CF02F0E4CFFE
:101C900001F0E4CF00F0E4CFD9FF1200C80EF66ED9
:101CA000230EF76E000EF86E0900F550056E090060
:101CB000F550066E055002E106503BE00900F55074
:101CC000006E0900F550016E0900F550026E090022
:101CD0000900F550E96E0900F550EA6E09000900A7
:101CE0000900F550036E0900F550046E0900090063
:101CF000F6CF07F0F7CF08F0F8CF09F000C0F6FFF5
:101D000001C0F7FF02C0F8FF035002E1045007E0F2
:101D10000900F550EE6E0306F8E20406F9D707C095
:101D2000F6FF08C0F7FF09C0F8FF0506C4E2060683
:101D3000C5D71200D9CFE5FFE1CFD9FF00C0E5FF3D
:101D400001C0E5FF02C0E5FF03C0E5FF04C0E5FFF9
:101D500005C0E5FF06C0E5FF020EDBCF00F0030E75
:101D6000DBCF01F0040EDBCF02F0050EDBCF03F07A
:101D7000060EDBCF04F0056A0450055C14E2055042
:101D80000324066E0650E56E7CEC11F0066EE12A27
:101D900006C0E5FF00C0E9FF01C0F3FF0250AEEC52
:101DA00011F0052AE9D70450E4CF06F0E4CF05F09E
:101DB000E4CF04F0E4CF03F0E4CF02F0E4CF01F08D
:101DC000E4CF00F0E4CFD9FF1200D9CFE5FFE1CF97
:101DD000D9FF800EE56E13EC11F0E12A010E706E52
:101DE000AE0E716E050E726E200E736E779E779C2E
:101DF000040E606E0F01506B0F01006B0F01016B41
:101E00000F01046B0F01056B0F01086B0F01096BCC
:101E10000F010C6B0F010D6B0F01106B0F01116B9C
:101E20000F01146B0F01156B0F01186B0F01196B6C
:101E30000F0119970F011C6B0F011D6B0F011D97EF
:101E4000000EE56E13EC11F0E12AE4CFD9FF120089
:101E5000D9CFE5FFE1CFD9FF00C0E5FF01C0E5FF25
:101E600002C0E5FF006E020EDBCF01F0030EDBCFF8
:101E700002F0AC6AAB6A00B0AC8800A202D0AC8CB5
:101E8000AB8C00A401D0AC8E00A602D0AB8801D0F0
:101E9000AB8A00A802D0AC8401D0AC949E9800AC70
:101EA00002D09D8A01D09D9A9E9A00AE02D09D8854
:101EB00001D09D980250B06E0150AF6E949C948EEC
:101EC000AC8AAB8EE4CF02F0E4CF01F0E4CF00F0B7
:101ED000E4CFD9FF1200E8CFE5FFD8CFE5FFE0CF90
:101EE000E5FFF3CFE5FFF4CFE5FFE9CFE5FFEACF6C
:101EF000E5FFFACFE5FFFBCFE5FFD9CFE5FFE1CF67
:101F0000D9FF00C0E5FF006AF2B4002A0050010AC0
:101F100003E159EC11F0F294E4CF00F0E4CFD9FFE3
:101F2000E4CFFBFFE4CFFAFFE4CFEAFFE4CFE9FF21
:101F3000E4CFF4FFE4CFF3FFE4CFE0FFE4CFD8FF3A
:101F4000E4CFE8FF1000D9CFE5FFE1CFD9FF00C013
:101F5000E5FF020EDBCF00F0030EDBCFA8FF00C0D1
:101F6000A9FFA69EA69CA684F29E550EA76EAA0E59
:101F7000A76EA682A6A202D00000FCD7A6A613D008
:101F8000450EC0EC11F0EBEC11F0006E0050FBE1DF
:101F9000520EC0EC11F0EBEC11F0006E0050FBE1C2
:101FA000520EC0EC11F0A694F28EE4CF00F0E4CF14
:101FB000D9FF1200D9CFE5FFE1CFD9FF00C0E5FF7F
:101FC00001C0E5FF02C0E5FF03C0E5FFE5EC0EF050
:101FD000006A016A0150800F800F02E1050E005C6B
:101FE00010E2970E0024026E000E0120036E02C064
:101FF000E9FF03C0EAFF000EEF6E002AD8B0012A05
:10200000E9D7F36AE86AE4CF03F0E4CF02F0E4CF63
:1020100001F0E4CF00F0E4CFD9FF1200D9CFE5FF03
:10202000E1CFD9FF00C0E5FF01C0E5FF02C0E5FF39
:1020300003C0E5FF04C0E5FF05C0E5FF020EDBCFEE
:1020400000F0005010E1D6CF00F0016AD7CF02F0C7
:10205000036A0250056E046A0450002605500122EE
:1020600001C0F3FF0050E4CF05F0E4CF04F0E4CF6B
:1020700003F0E4CF02F0E4CF01F0E4CF00F0E4CFCE
:10208000D9FF1200D9CFE5FFE1CFD9FF00C0E5FFAE
:1020900001C0E5FF02C0E5FF03C0E5FF020EDBCF94
:1020A00000F0030EDBCF01F0040EDBCF02F0005096
:1020B000011008E10250C0EC11F0EBEC11F0036EDE
:1020C0000350FBE10050010A02E1015001E002D09F
:1020D00002C0C9FFE4CF03F0E4CF02F0E4CF01F087
:1020E000E4CF00F0E4CFD9FF1200D9CFE5FFE1CF74
:1020F000D9FF00C0E5FF01C0E5FF02C0E5FF020E09
:10210000DBCF00F0030EDBCF01F00050011006E141
:102110009E9A45EC11F0026E02500BD00050010A5D
:1021200002E1015001E004D0C7A002D0C95001D0A3
:10213000E86AE4CF02F0E4CF01F0E4CF00F0E4CFAE
:10214000D9FF1200D9CFE5FFE1CFD9FF00C0E5FFED
:1021500001C0E5FF020EDBCF00F0030EDBCF01F084
:102160000050011006E19EAA02D0010E0FD0E86ACD
:102170000DD00050010A02E1015001E006D0C7A0D5
:1021800002D0010E03D0E86A01D0E86AE4CF01F082
:10219000E4CF00F0E4CFD9FF1200D9CFE5FFE1CFC3
:1021A000D9FF00C0E5FF01C0E5FF02C0E5FF03C0A5
:1021B000E5FF020EDBCF00F0030EDBCF01F0015094
:1021C000026E036A0250D76E0050D66EE4CF03F061
:1021D000E4CF02F0E4CF01F0E4CF00F0E4CFD9FF88
:1021E0001200D9CFE5FFE1CFD9FF00C0E5FF01C064
:1021F000E5FF020EDBCF00F0030EDBCF01F0005055
:10220000011009E1EBEC11F0006E005002E0E86A09
:1022100003D0010E01D0E86AE4CF01F0E4CF00F072
:10222000E4CFD9FF1200D9CFE5FFE1CFD9FF00C03D
:10223000E5FF01C0E5FF020EDBCF00F01F0E6F16B9
:1022400000506F12E00E6F14016E01500018FAE199
:10225000E4CF01F0E4CF00F0E4CFD9FF1200E8AE04
:1022600006D0F3CFEAFFEE50EECFF3FF1200E8BC4A
:102270000BD0E9CFF6FFF3CFF7FFF86E0900F5506A
:102280000900F5CFF3FF12001200F00E0001AF15A8
:10229000AF6FABAC04D0AF91ABA001D0AF81ABA41A
:1022A00002D00001AF85ABA202D00001AF87AE50D3
:1022B0001200D9CFE5FFE1CFD9FF00018951E56ECA
:1022C000000EE56E000EE56E42EC10F0030EE12606
:1022D000E4CFD9FF1200E8AE04D0F3CFEAFFEE500E
:1022E0001200E8BC08D0E9CFF6FFF3CFF7FFF86E95
:1022F0000900F55012001200D9CFE5FFE1CFD9FF58
:10230000020EDBCFA9FFA69CA69EA680A850E4CF14
:10231000D9FF1200D9CFE5FFE1CFD9FFF28AF184CE
:10232000F28EF36A010EE4CFD9FF120017EEFFF030
:1023300027EEFFF0F86AA68EA69C4EEC0EF0FEEC9F
:102340000AF0FFD7E8AE07D0F3CFEAFFE4CFEEFF05
:10235000F4CFEEFF1200E8AC12001200E8AE05D098
:10236000F3CFEAFFE4CFEEFF1200E8AC1200120058
:10237000617B008097008000000102030405AA0031
:10238000ACAC04D0AC900001AFB3AC80AD6E120029
:10239000D9CFE5FFE1CFD9FFE4CFD9FF1200D9CFE4
:1023A000E5FFE1CFD9FFE4CFD9FF1200D9CFE5FF98
:1023B000E1CFD9FFE4CFD9FF1200D9CFE5FFE1CFBC
:1023C000D9FFE4CFD9FF12000100702300007B0089
:0E23D000000010000000000EACA2010F120071
:020000040030CA
:0E000000FFF2FFFEFFFFBBFFFFFFFFFFFFFF52
:00000001FF
